:100000004129A0007F39201B803C0920A01B003C17
:1000100008008A01820700340334063409340C34A2
:1000200010341334163419341C341F34223425345C
:1000300028342B342E3431343334363439343C3490
:100040003F3441344434473449344C344E345134D1
:100050005334553458345A345C345E34603462342A
:100060006434663468346A346B346D346F3470349D
:1000700071347334743475347634783479347A3432
:100080007A347B347C347D347D347E347E347E34EB
:100090007F347F347F347F34A4002508A402031CFE
:1000A000A5032708A602031CA7033709A2003509E8
:1000B000A300A20A0319A30A4130A900AC01AD01B3
:1000C000AE01AF01A8013608840034098E208413E4
:1000D0003D212408AC070318AD0A2508AD07260802
:1000E000AE070318AF0A2708AF072D080120803E8E
:1000F000A1002F080120803EA107210CA8070008BD
:100100003404031C34068000290303194130A9007C
:100110000319A20A0319A30F68283C298417800534
:100120003C299620B4000408B6000800A800053059
:10013000A8190530840000308A0028080739820792
:100140000134023404340834103420344034803410
:100150000F39A0000310A00DA00D1F08E0392004E6
:1001600001389F000030A1003230DD209F149F181D
:10017000B7281E08A10083161E083C2983169B0081
:100180001C141A083C2983169A001C1555309D0032
:10019000AA309D009C149C18CB281C113C29A3015B
:1001A000A200FF30A207031CA307031C3C29033055
:1001B000A100E630DD20D128A101FC3EA000A1096C
:1001C000031CE828FF300000A0070318E328A0075D
:1001D0000000A10FE22808000310A00DA10DFF3EB2
:1001E0000318EC2820083C290310A10CA00CFF3EAA
:1001F0000318F42820083C29A101A301A200033020
:100200000B29A101A301A20001300B29A101A30127
:10021000A20006300B29A80023082102031D122981
:100220002208200204300318013003190230280587
:10023000031DFF303C290038031DFF300405031D5A
:10024000FF303C290404031DFF303C291030A80076
:10025000A101A001A70CA60C031C34292208A007A9
:1002600023080318230FA107A10CA00CA50CA40CB4
:10027000A80B2A2924083C298313031383120000A6
:10028000080089309F00E901FE30BE20EA00FF30FF
:10029000BE20E7000230A820DB002108DC005B085C
:1002A000A0005C08A100A30125300321DD005B084C
:1002B000A0005C08A100A3016E300821DF005D08EA
:1002C00084005F081B21DF00E0005F086004031961
:1002D00081296A08003C031D70290130EA00752954
:1002E0006A08013C031D7529EA0100309120E830BD
:1002F000B7000330B5000630A700A500A430A60063
:100300004C205B08A0005C08A1000130A300003075
:100310000321DD005B08A0005C08A1000130A30000
:1003200049300821DF005D0884005F081B21DF00E1
:10033000E0005F0860040319C729FE30BE20EE000C
:100340006E08003C031DAD290130EE008316FE301F
:100350009B0083126E08C320B8296E08013C031D60
:10036000B829EE018316FE309B0083126E08C3206D
:10037000FE30BE20EA0000309120E830B7000330A4
:10038000B5000630A700A500A430A6004C205B08ED
:10039000A0005C08A100A3016E300321DD005B0812
:1003A000A0005C08A100A301B6300821DF005D08B1
:1003B00084005F081B21DF00E0005F086004031970
:1003C0000C2AFF30BE20EE006E084B3C031DF129C5
:1003D0007830EE008316FF309B0083126E08C32036
:1003E000FD296E08783C031DFD294B30EE00831675
:1003F000FF309B0083126E08C320FF30BE20E70051
:1004000000309120E830B7000330B5000630A70077
:10041000A500A430A6004C200230A820DB00210853
:10042000DC000A30CF205B08A0005C08A100A3011B
:1004300025300321031D0C2A0130EC006A08003C22
:10044000031D232AB8016A08013C031D292A0E3026
:10045000B800FF30B9000230A820DB002108DC0022
:10046000E6015B08A0005C08A100A301253008217B
:10047000031D3B2A3E220A30CF202B2A5B08A00016
:100480005C08A1000330A30092300321DD005B086B
:10049000A0005C08A1000330A300FF300821DF00AA
:1004A0005D0884005F081B21DF00E0005F08600436
:1004B00003195E2A0130E300EE242E245B08A0001D
:1004C0005C08A1000330A30049300321DD005B0874
:1004D000A0005C08A1000330A30092300821DF00D7
:1004E0005D0884005F081B21DF00E0005F086004F6
:1004F00003197E2A0230E300EE242E245B08A000BC
:100500005C08A1000230A300FF300321DD005B087E
:10051000A0005C08A1000330A30049300821DF00DF
:100520005D0884005F081B21DF00E0005F086004B5
:1005300003199E2A0330E300EE242E245B08A0005A
:100540005C08A1000230A300B6300321DD005B0887
:10055000A0005C08A1000230A300FF300821DF00EA
:100560005D0884005F081B21DF00E0005F08600475
:100570000319BE2A0430E300EE242E245B08A000F9
:100580005C08A1000230A3006D300321DD005B0890
:10059000A0005C08A1000230A300B6300821DF00F3
:1005A0005D0884005F081B21DF00E0005F08600435
:1005B0000319DE2A0530E300EE242E245B08A00098
:1005C0005C08A1000230A30025300321DD005B0898
:1005D000A0005C08A1000230A3006D300821DF00FC
:1005E0005D0884005F081B21DF00E0005F086004F5
:1005F0000319FE2A0630E300EE242E245B08A00037
:100600005C08A1000130A300DB300321DD005B08A2
:10061000A0005C08A1000230A30025300821DF0003
:100620005D0884005F081B21DF00E0005F086004B4
:1006300003191E2B0730E300EE242E245B08A000D4
:100640005C08A1000130A30091300321DD005B08AC
:10065000A0005C08A1000130A300DB300821DF000E
:100660005D0884005F081B21DF00E0005F08600474
:1006700003193E2B0830E300EE242E245B08A00073
:100680005C08A1000130A30049300321DD005B08B4
:10069000A0005C08A1000130A30091300821DF0018
:1006A0005D0884005F081B21DF00E0005F08600434
:1006B00003195E2B0930E300EE242E245B08A00012
:1006C0005C08A1000130A30000300321DD005B08BD
:1006D000A0005C08A1000130A30049300821DF0020
:1006E0005D0884005F081B21DF00E0005F086004F4
:1006F00003197E2B0A30E300EE242E245B08A000B1
:100700005C08A100A301B6300321DD005B08A00056
:100710005C08A1000130A30000300821DF005D0863
:1007200084005F081B21DF00E0005F0860040319FC
:100730009D2B0B30E300EE242E245B08A0005C0808
:10074000A100A3016E300321DD005B08A0005C085E
:10075000A100A301B6300821DF005D0884005F0816
:100760001B21DF00E0005F0860040319BB2B0C3085
:10077000E300EE242E245B08A0005C08A100A30186
:1007800025300321DD005B08A0005C08A100A30167
:100790006E300821DF005D0884005F081B21DF0048
:1007A000E0005F0860040319D92B0D30E300EE244C
:1007B0002E240230A820DB002108DC00E60A6608AF
:1007C000A00064300121DD005B08A0005C08A100EE
:1007D000A30125300321DF005D0884005F081B2191
:1007E000DF00E0005B08A0005C08A100A3016E3000
:1007F0000821E1005F086004840061081B21E1001A
:10080000E200610862040319062C4A276908003CCB
:10081000031D222C6608A000C8300121DD005B0802
:10082000A0005C08A100A3016E300321DF005D0879
:1008300084005F081B21DF00E0005F0860040319EB
:10084000222C51240A30CF205B08A0005C08A100B4
:10085000A30125300321031DD92B08006C08223C7D
:10086000031DFF30FF3ADD006908013C031DFF3026
:10087000FF3ADF005D0884005F082221DF00E0000E
:100880005F0860040319452C08006C08383E84009A
:1008900063088000EC0A6C08383E8400FF3080005A
:1008A0000800003091204B30B700B5010630A7009A
:1008B000A500A430A6004C20FF306C07DD00FF30FF
:1008C0000318013EDE005D08383E8400FF308000E2
:1008D000EC010730630203187D2CFF306307DD0055
:1008E000FF300318013EDE002230A600A7015D089C
:1008F000A2005E08A3002621EF006308A0000730D5
:10090000FC20DD006308A0000C300621DF005D083C
:1009100084005F081B21DF00E0005F08600403190A
:10092000A12CF9306307DD00FF300318013EDE0023
:100930002230A600A7015D08A2005E08A3002621C0
:10094000EF006C08383E84000008DD005D08FF3CC5
:10095000031DDF2C0F30E400A8276F0883169B00CF
:1009600083126408C3200130EC006A08003C031DB8
:10097000BA2CB8016A08013C031DC02C0E30B80027
:10098000FF30B90000309120E830B7000330B500E7
:100990000530A700A500DC30A6004C200230A820BE
:1009A000DB002108DC000A30CF205B08A0005C08D7
:1009B000A100A30125300321031DCE2C08006C08E3
:1009C000383E84000008E400A8276F0883169B00C7
:1009D00083126408C320EC0AEF0AA12C6908003CCA
:1009E000031DF32C462D6308A0000130FC20DD0020
:1009F0006308A00006300621DF005D0884005F0860
:100A00001B21DF00E0005F0860040319172DFF3091
:100A10006307DD00FF300318013EDE002230A60030
:100A2000A7015D08A2005E08A3002621ED0063086F
:100A3000A0000730FC20DD006308A0000C30062178
:100A4000DF005D0884005F081B21DF00E0005F0815
:100A5000600403193B2DF9306307DD00FF300318F4
:100A6000013EDE002230A600A7015D08A2005E085C
:100A7000A3002621ED000D306302031C402D080069
:100A80006308E5006D08BE20E400C1276A08013C48
:100A900003193A2E63080F3C031D4F2D080063080D
:100AA000003C031D542DEA016308013C031D652D24
:100AB000003091206708B700B5018430A6000330EC
:100AC000A7000230A500BC304C206308023C031D87
:100AD000762D003091206708B700B5014C30A60094
:100AE0000430A7000230A500BC304C206308033C52
:100AF000031D872D003091206708B700B5014C30E9
:100B0000A6000430A7000330A50084304C20630801
:100B1000043C031D982D003091206708B700B501F3
:100B20001430A6000530A7000230A500BC304C20D0
:100B30006308053C031DA92D003091206708B7000C
:100B4000B5011430A6000530A7000330A50084309D
:100B50004C206308063C031DBA2D00309120670825
:100B6000B700B5011430A6000530A7000430A50079
:100B70004C304C206308073C031DCB2D00309120E6
:100B80006708B700B501DC30A6000530A7000230C9
:100B9000A500BC304C206308083C031DDC2D003050
:100BA00091206708B700B501DC30A6000530A7002A
:100BB0000330A50084304C206308093C031DED2D53
:100BC000003091206708B700B501DC30A600053081
:100BD000A7000430A5004C304C2063080A3C031DDC
:100BE000FE2D003091207830B700B501A430A6006A
:100BF0000630A7000430A5004C304C2063080B3CA5
:100C0000031D0F2E003091206708B700B501DC30BE
:100C1000A6000530A7000530A50014304C2063085D
:100C20000C3C031D202E003091206708B700B50151
:100C3000A430A6000630A7000530A500DC304C200B
:100C400063080D3C031D302E00309120E830B700C2
:100C50000330B5000A30A700A5002830A6004C20BC
:100C600063080E3C031D362E0130EA006A08003C82
:100C70000319262F63080F3C031D3F2E080063084D
:100C8000003C031D442EEA016308013C031D552E60
:100C9000003091206708B700B501B930A6000430D4
:100CA000A7000230A500B9304C206308023C031DA8
:100CB000662E003091206708B700B5013830A600D5
:100CC0000530A7000230A500B9304C206308033C72
:100CD000031D772E003091206708B700B501C5309D
:100CE000A6000530A7000230A500B9304C206308EB
:100CF000043C031D882E003091206708B700B50121
:100D0000B930A6000430A7000330A50002304C2003
:100D10006308053C031D992E003091206708B70039
:100D2000B5013830A6000530A7000330A500023019
:100D30004C206308063C031DAA2E00309120670852
:100D4000B700B501C530A6000530A7000330A500E7
:100D500002304C206308073C031DBB2E003091205D
:100D60006708B700B501B930A6000430A70003300A
:100D7000A50054304C206308083C031DCC2E0030E5
:100D800091206708B700B5013830A6000530A700EC
:100D90000330A50054304C206308093C031DDD2EB0
:100DA000003091206708B700B501C530A6000530B6
:100DB000A7000330A50054304C2063080A3C031DF3
:100DC000EE2E003091206708B700B501B930A600BB
:100DD0000430A7000330A500AD304C2063080B3C65
:100DE000031DFF2E003091206708B700B501383091
:100DF000A6000530A7000330A500AD304C206308E5
:100E00000C3C031D102F003091206708B700B5017E
:100E1000C530A6000530A7000330A500AD304C203A
:100E200063080D3C031D202F00309120E830B700EF
:100E30000330B5000A30A700A5002830A6004C20DA
:100E400063080E3C031D262F0130EA0063080D3CA9
:100E5000031DFF30FF3ADD006908013C031DFF3030
:100E6000FF3ADF005D0884005F081B21DF00E0001F
:100E70005F0860040319402F0530A300DC30D02048
:100E80006908003C031D452F0800ED0A6708CF20C4
:100E9000422D08006908013C031D692FE9016B0818
:100EA000EA00E601003091204B30B700B501063072
:100EB000A700A500A430A6004C20003091204B30A4
:100EC000B700B5010530A700A5001430A6004C20DE
:100ED000972F6908003C031D972F0130E9006A082D
:100EE000EB00E601003091204B30B700B501053032
:100EF000A700A5001430A6004C20003091204B30F4
:100F0000B700B5010630A700A500A430A6004C200C
:100F10000130EC006A08003C031D8F2FB8016A08FD
:100F2000013C031D952F0E30B800FF30B900023090
:100F3000A820DB002108DC000A30CF205B08A000DD
:100F40005C08A100A30125300321031D972F080091
:100F500007306302031CB32F0F30E8006408A000C1
:100F60000430EF20E400073063020318B92FF0309B
:100F7000E8006F08BE20EE006808EE056E08E40485
:100F800008006508A0000730FC20DD006508A0000F
:100F90000C300621DF005D0884005F081B21DF00A4
:100FA000E0005F0860040319DC2F6408A000A101C1
:100FB0000430F720E300F52F6508A0000130FC2085
:100FC000DD006508A00006300621DF005D08840012
:100FD0005F081B21DF00E0005F0860040319F52FA4
:0C0FE0000F30E80064086805E30008001A
:02400E00E2309E
:02420000FF00BD
:02424400FF0079
:02428800FF0035
:0242CC00FF00F1
:02431000FF00AC
:02435400FF0068
:0443FC0000004B0072
:00000001FF
